:100000000C9464000C9481000C9481000C942307E0
:100010000C9481000C9481000C9481000C94F606E1
:100020000C9481000C9481000C9481000C9481004C
:100030000C9481000C9481000C9481000C9481003C
:100040000C9481000C9481000C9481000C9481002C
:100050000C9481000C9481000C942104A8EA802A5D
:100060000040000A510A084059551801111E111B81
:10007000500B411B411F1101511F511B000000007B
:100080000880001A204000000000510F91394114EF
:100090009131411E410E411D500F802010154886A0
:1000A0004014780570855115510E5195518E21904F
:1000B00081205015484450C528C0282009504114BB
:1000C000208011110000001011241FBECFEFD4E0DA
:1000D000DEBFCDBF11E0A0E0B1E0E0EEF6E102C08E
:1000E00005900D92A03DB107D9F712E0A0EDB1E067
:1000F00001C01D92A531B107E1F70E941C020C94CA
:100100006E0B0C940000EF92FF920F931F93DF93FE
:10011000CF93CDB7DEB7C955D0400FB6F894DEBF48
:100120000FBECDBF8C0145E050E060E071E00E9461
:100130007F08009711F58091D3019091D401009729
:1001400011F00E940908C80105960E946108809379
:10015000D00190E0880F991F0E945F078093D30120
:100160009093D4018091D00190E00E94790581E0C4
:100170008093A80121E030E06DC044E050E066E0EB
:1001800071E0C8010E947F08009719F420E030E078
:1001900061C044E050E06BE071E0C8010E947F085C
:1001A000009761F580E191E00E946C01C80104961E
:1001B0000E946108E82EC80107960E946108F82E87
:1001C00090E09F938F938E2D90E09F938F938DE27D
:1001D00091E09F938F938E010F5F1F4F1F930F939B
:1001E0000E949508C8010E946C016F2D8E2D0E94FF
:1001F0007C058091D101282F30E024C0DE015A9681
:10020000E5E4F1E082E101900D928150E1F7FE0119
:10021000BC968EE2DF011D928A95E9F71F930F933A
:100220008E01065E1F4F1F930F938EE391E09F9305
:100230008F931F930F930E949508C8010E946C0131
:1002400020E030E08DB79EB708960FB6F8949EBFB9
:100250000FBE8DBFC901C75ADF4F0FB6F894DEBF7E
:100260000FBECDBFCF91DF911F910F91FF90EF9007
:1002700008950E94B8010E949D010E94C2030E943D
:10028000DE020E94B2060E941A0708958091C00003
:10029000881F8827881F08958091C600089580933D
:1002A000C6000FB607FE0EC020E030E002C02F5F90
:1002B0003F4F8091C00086FD09C087E2203138079A
:1002C000B1F704C08091C00086FFFCCF8091C000D0
:1002D00080648093C00008950F931F93CF93DF93A2
:1002E0008C01C0E0D0E0F801EC0FFD1F8081882375
:1002F00031F021960E944F01C034D105A1F7DF9162
:10030000CF911F910F9108950F931F93CF93DF9378
:100310008C01C0E0D0E002C00E944F01F801EC0F58
:10032000FD1F8491882321F02196CD33D105A1F7BB
:10033000DF91CF911F910F910895E1E6F0E080E801
:10034000808392E090831092C5008CE08093C4007B
:100350009093C00088E18093C10086E08093C20042
:10036000789480E580936C0080E88CBB8DBB089509
:1003700080E88093610083E08093610010927000B8
:1003800088E08093B60088EC8093B30010926E00F2
:1003900081E0809381008093B0002091B60080912D
:1003A000B60090E08470907030E021703070822B45
:1003B000932B892B91F780E090E020E335E7F9015A
:1003C0003197F1F701968A309105C9F74FEF51E067
:1003D000F89446BB47BB109285001092840010929F
:1003E000B20087B38823E9F310928100789486B332
:1003F0008823B9F49091840080918500382F20E003
:10040000B901690F711DCB0178E18B36970724F094
:1004100080916600815008C0885E974114F081E0A9
:1004200006C0809166008F5F8093660080E05093E5
:100430008100882369F208952F923F924F925F9234
:100440006F927F928F929F92AF92BF92CF92DF92E4
:10045000EF92FF920F931F93DF93CF93CDB7DEB749
:10046000C258D0400FB6F894DEBF0FBECDBF0E9479
:100470003901FF245E010894A11CB11C71E4C72E50
:10048000D12CCC0EDD1E64E4662E712C812C912CB7
:10049000CE018B5B9F4FCF57DF4F99838883C15825
:1004A000D0405CE3E52E4EE9242E41E0342E34EAC0
:1004B000432E31E0532E11C01082C5010E948300EB
:1004C0008093D101198208C09FE39F1530F41982EF
:1004D00085E891E00E946C01FF248091C00087FFB5
:1004E00067C08091C600F501EF0DF11D8083F39484
:1004F000EF2DF0E03197EA0DFB1D80818A3021F766
:10050000DBCFF894F6016082718282829382CF57AA
:10051000DF4FE881F981C158D0408E2D11928A9524
:10052000E9F700E010E01FC0C801880F991FE091B3
:10053000D301F091D401E80FF91F808191819F933D
:100540008F93DF92CF923F922F92DF92CF920E94B1
:1005500095080F5F1F4FEDB7FEB738960FB6F894AA
:10056000FEBF0FBEEDBF8091D00190E008171907C4
:10057000DCF21092D20178948091A801813021F4AC
:1005800061E0C6010E94FE04DF92CF925F924F921B
:10059000DF92CF920E949508C6010E946C018DB730
:1005A0009EB706960FB6F8949EBF0FBE8DBF95CF2F
:1005B0008091D201813009F090CFA3CF759A749ABF
:1005C0006C9A6D9A8FEF8093BA008AE28093B8009C
:1005D00080EF8093B90008958091DA0108958093A7
:1005E000B90033E09BE222E0832F8A95F1F79093E4
:1005F000B800649BFECF822F8A95F1F79093B800E4
:100600008091B90086FFF0CF83E08A95F1F7809161
:10061000BA009FEF9093BA006D9A0895749A749BF4
:10062000FECF93E0892F8A95F1F7759882E08A953D
:10063000F1F77498759A8091B90087FF02C081E044
:1006400008959093DA0180E008957598749A649BF8
:10065000FECF82E08A95F1F7759A83E08A95F1F7EB
:100660008091B90085FF02C081E0089584E0809305
:10067000DA0180E00895CF92DF92EF92FF920F931C
:100680001F93CF93DF938C01E62E9091DA01892F8F
:1006900081608093DA01F801808180FD03C093605E
:1006A0009093DA010E940E03882309F452C0E801F6
:1006B000FE2CCC24CA94DD24D3948091DA0183707B
:1006C00081F1749888818093BA0080EF0E94EF02D4
:1006D0006D988EEF0E94EF029091DA0180FF09C0C1
:1006E00090FF02C081E001C082E08093DA0180E0E7
:1006F00030C0892F8570843079F4F8018081816061
:100700008083D092DA010E940E03882319F0E80159
:10071000FE2C18C08AE0E9CF21969E7F9093DA01E3
:1007200011C06D9880EF0E94EF028883F1E0FF1600
:1007300019F4C092BA0002C01092BA0021968EEF4E
:100740000E94EF02FA9409F0B8CF0E9425038111AC
:1007500081E0DF91CF911F910F91FF90EF90DF909B
:10076000CF9008951092DA010E943B030895FC0196
:1007700080818E7F808384E08093DA01CF010E94A4
:100780003B030895ECEDF1E0119281E0E03FF807C2
:10079000D9F78FE08093E70087EB8093E50087E04F
:1007A0008093E60080EC8093E4008091E400886010
:1007B0008093E4001092D5010895982F6630B0F52B
:1007C0008A52813518F040E050E00CC0913608F0B4
:1007D0009F7D9A52E92FF0E0EE0FFF1FE45AFF4F82
:1007E00045915491862F90E0DC01A170B07060FDBE
:1007F00002C090EF01C09FE06695E62FF0E0E45262
:10080000FE4F30E0242F2F7084E0569547958A954F
:10081000E1F7109711F02295207F80818923282B02
:1008200020833F5F343011F03596ECCF089581116D
:100830008FEFECEDF1E0819391E0E03FF907D9F71C
:1008400008951F920F920FB60F921124EF92FF920C
:100850000F931F932F933F934F935F936F937F93C8
:100860008F939F93AF93BF93CF93DF93EF93FF93B8
:100870000091A90101500093A9018091DB01882317
:1008800071F0002371F48091D601882321F481E076
:100890008093D50106C081508093D60102C010928A
:1008A00009028091D501813009F053C0E090D70151
:1008B000FF2410E0C0E0D0E06C2F8091090299275E
:1008C00087FD90958C0F9D1F97FD16C01123A1F4F5
:1008D00080910902992787FD9095FE01E051FE4F16
:1008E000E80FF91F8081F82EFF1CFF24FF1C8F7773
:1008F00021F41C2F1F5F01C080E2FF2021F094E053
:100900009E1508F480E20E94DD032196C630D105D1
:1009100099F6ACEEB0E0FD01E051FF4F80818D9380
:1009200081E0A030B807B9F78091D801882321F081
:1009300081E08093F40002C01092F400113011F4B1
:100940008AEF03C0809109028F5F809309021092A1
:10095000D501002319F483E08093A9018091D70188
:100960008A3019F41092D70103C08F5F8093D701AA
:10097000FF91EF91DF91CF91BF91AF919F918F91B7
:100980007F916F915F914F913F912F911F910F91A7
:10099000FF90EF900F900FBE0F901F901895382F7B
:1009A000292F8091D5018823E1F7A0EFB1E0832FB3
:1009B000922FFC0101C02D938E2F831B24912223A3
:1009C00029F0319692E0A930B907A9F790E0FC012F
:1009D000E051FE4F108207974CF081E08093DB01DD
:1009E0001092090283E08093D60104C01092DB01CB
:1009F0001092090281E08093D5010895482F292F94
:100A00008091D5018823E1F7A0EFB1E0842F922FE8
:100A10009C01F90101C02D938E2F841B208122237C
:100A200029F0319692E0A930B907A9F790E0FC01CE
:100A3000E051FE4F108207974CF081E08093DB017C
:100A40001092090283E08093D60104C01092DB016A
:100A50001092090281E08093D5010895893128F42C
:100A6000E82FF0E0E051FE4F60830895E0EFF1E001
:100A7000119282E0E930F807D9F708958093D80100
:100A80000895982F8091D5018823E1F76093DB01C9
:100A9000109209029093D50108951092D7010895FC
:100AA000982FE0EFF1E0119282E0E930F807D9F7F2
:100AB00081E48093F00182E48093F10183E48093E8
:100AC000F20184E48093F30185E48093F40186E4E9
:100AD0008093F5018091D5018823E1F71092DB0125
:100AE0001092090281E08093D5019F709093E700F6
:100AF00008958093D0010895DF92EF92FF920F93B3
:100B00001F93DF93CF93CDB7DEB764970FB6F894FA
:100B1000DEBF0FBECDBFD62EF82EFF0CDD0C8D2D07
:100B200090E09F938F938F2D90E09F938F938BEA0C
:100B300091E09F938F938E010F5F1F4F1F930F9331
:100B40000E949508C8010E946C0180EEF80E0AE030
:100B500012E0F0920A0210920B0280EA80930C02DB
:100B600063E0C8010E94B2038DE0E82E8E2D8A95C5
:100B7000F1F7F0920A0210920B028AEA80930C02BB
:100B800063E0C8010E94B2038E2D8A95F1F7F092BE
:100B90000A0210920B0285EA80930C0263E0C801FE
:100BA0000E94B2038E2D8A95F1F7F0920A021092FC
:100BB0000B0290EED90ED0920C0263E0C8010E94A5
:100BC000B203EA94F1F78DB79EB708960FB6F89482
:100BD0009EBF0FBE8DBF64960FB6F894DEBF0FBEEA
:100BE000CDBFCF91DF911F910F91FF90EF90DF90DC
:100BF0000895880F8F5180930A0210920B0262E0D1
:100C00008AE092E00E94B20380910B0208950E9454
:100C1000F90581E008950F931F93182F062F90E098
:100C20009F938F9389EB91E09F938F930E949508F8
:100C3000110F105210930A0210920B0200930C0233
:100C400063E08AE092E00E94B2030F900F900F9051
:100C50000F901F910F9108951F93CF93DF93182F3B
:100C6000C0E0D0E005C0612F8C2F0E940B062296B9
:100C70008091D00190E0C817D907ACF3C1E0D0E073
:100C800005C0612F8C2F0E940B0622968091D00107
:100C900090E0C817D907ACF3DF91CF911F91089569
:100CA000DF92EF92FF920F931F93082F0E94F90596
:100CB000D02EDD0C81EED80E9AE0E92E92E0F92ECE
:100CC000D0920A0282E080930B0262E0C7010E9488
:100CD000B20310910B0200E0D0920A0283E08093ED
:100CE0000B0262E0C7010E94B20320910B0230E0C8
:100CF000202B312BC9011F910F91FF90EF90DF90B6
:100D000008951F93182F0E940B0684EF91E001971E
:100D1000F1F7812F0E9450061F910895EF92FF92E4
:100D20000F931F93CF93DF93F82EE92E9C01890137
:100D3000C0E0D0E008C08C2F0E945006F8018193DB
:100D400091938F0121968091D00190E0C817D90727
:100D500094F38F2D9E2DDF91CF911F910F91FF90D6
:100D6000EF900895109285001092840088EA91E631
:100D700090938900809388008AE08093810082E0CC
:100D800080936F00089580910F0290911002019658
:100D90009093100280930F029091D101913029F528
:100DA0008091D9018F5F8093D901833258F01092DE
:100DB000D9018091A801813019F41092A80102C0D4
:100DC0009093A80181E50E942C0680E18A95F1F7B5
:100DD0008091D3019091D4010E948E069093D4010A
:100DE0008093D30181E08093D20108951F920F92E6
:100DF0000FB60F9211242F933F934F935F936F93EE
:100E00007F938F939F93AF93BF93EF93FF930E9432
:100E1000C306FF91EF91BF91AF919F918F917F9109
:100E20006F915F914F913F912F910F900FBE0F9057
:100E30001F90189584B114B82C9A80E180936C00AF
:100E4000EF9AE79A08951F920F920FB60F9211240E
:100E50002F933F934F935F936F937F938F939F93C2
:100E6000AF93BF93EF93FF938091D101813019F439
:100E70001092D10103C081E08093D1018091D00113
:100E8000882359F484E08093D00188E090E00E94A8
:100E90005F078093D3019093D401E79AFF91EF917C
:100EA000BF91AF919F918F917F916F915F914F9182
:100EB0003F912F910F900FBE0F901F901895CF93D9
:100EC000DF93BC018230910510F462E070E0A091E4
:100ED0001302B0911402ED01E0E0F0E040E050E0D8
:100EE00021C0888199818617970769F48A819B813F
:100EF000309719F09383828304C0909314028093F7
:100F00001302FE0134C06817790738F44115510502
:100F100019F08417950708F4AC01FE018A819B81C2
:100F20009C01E9012097E9F641155105A9F1CA0193
:100F3000861B970B049708F4BA01E0E0F0E02AC0A2
:100F40008D919C91119784179507F9F46417750793
:100F500081F412968D919C911397309719F0938399
:100F6000828304C09093140280931302FD01329691
:100F70004CC0CA01861B970BFD01E80FF91F619356
:100F8000719302978D939C9340C0FD018281938160
:100F90009C01D9011097A1F6809111029091120243
:100FA000892B41F48091CC019091CD019093120254
:100FB000809311024091CE015091CF01411551050E
:100FC00041F44DB75EB78091CA019091CB01481BA7
:100FD000590B2091110230911202CA01821B930B0E
:100FE0008617970780F0AB014E5F5F4F8417950718
:100FF00050F0420F531F5093120240931102F90117
:101000006193719302C0E0E0F0E0CF01DF91CF91F6
:101010000895CF93DF93009709F450C0EC01229715
:101020001B821A82A0911302B0911402109709F149
:1010300040E050E0AC17BD0708F1BB83AA83FE0176
:1010400021913191E20FF31FAE17BF0779F48D9113
:101050009C911197280F391F2E5F3F4F39832883AA
:1010600012968D919C9113979B838A83411551050C
:1010700071F4D0931402C093130220C012968D9184
:101080009C911397AD01009711F0DC01D3CFFA01C9
:10109000D383C28321913191E20FF31FCE17DF0773
:1010A00069F488819981280F391F2E5F3F4FFA011B
:1010B000318320838A819B8193838283DF91CF91C7
:1010C0000895FC0188279927E89421912032E9F3BB
:1010D000293010F02E30C8F32B3241F02D3239F484
:1010E000689404C00E948D08820F911D21912053A5
:1010F0002A30C0F31EF4909581959F4F0895FB010F
:10110000DC014150504030F08D910190801919F46C
:101110000020B9F7881B990B08957AE0979F902DCE
:10112000879F802D910D11240895AEE0B0E0EBE98A
:10113000F8E00C94450B0D891E8986E08C831A8398
:1011400009838FEF9FE79E838D83CE014996AC0183
:101150006F89788DCE0101960E94B8082F8138855D
:10116000020F131FF80110822E96E4E00C94610B1D
:10117000ABE0B0E0EEEBF8E00C94370B3C012B0158
:101180005A01FC0117821682838181FD03C06FEF33
:101190007FEFC8C19AE0892E1E010894211C311CE2
:1011A000F3012381F20123FD859123FF81912F011A
:1011B000882309F4B4C1853239F423FD859123FFD6
:1011C00081912F01853229F4B30190E00E94AD0A8C
:1011D000E7CF982FDD24CC249924FFE1FD15D0F032
:1011E0009B3269F09C3228F4903259F0933291F49A
:1011F0000EC09D3249F0903369F441E024C052E0C2
:10120000D52A84E0D82A28C098E0D92A25C0E0E170
:10121000DE2A22C0D7FC29C0892F80538A3070F47F
:10122000D6FE05C0989C902C1124980E15C0C89C21
:10123000C02C1124C80EF0E2DF2A0EC09E3229F421
:10124000D6FC6DC140E4D42A07C09C3619F450E89E
:10125000D52A02C0983649F4F20123FD959123FF67
:1012600091912F01992309F0B8CF892F85548330AC
:1012700018F08052833038F444E050E0A40EB51EDC
:101280005FE359830FC0933631F0933779F093358C
:1012900009F056C020C0F5018081898342E050E00A
:1012A000A40EB51E710101E010E012C0F501E0804E
:1012B000F180D6FC03C06FEF7FEF02C0692D70E0B4
:1012C00042E050E0A40EB51EC7010E94A20A8C01A4
:1012D0005FE7D52214C0F501E080F180D6FC03C0A1
:1012E0006FEF7FEF02C0692D70E042E050E0A40E86
:1012F000B51EC7010E94970A8C0150E8D52AD3FE7B
:1013000007C01AC0B30180E290E00E94AD0ACA94FF
:101310008C2D90E008171907A8F30EC0F701D7FC31
:101320008591D7FE81917F01B30190E00E94AD0AC3
:10133000C110CA94015010400115110579F7ECC095
:10134000943611F0993671F5D7FE08C0F501E080AA
:10135000F1800281138144E050E00AC0F5018081F0
:1013600091817C010027F7FC0095102F42E050E0AE
:10137000A40EB51E5FE6D52217FF0AC01095009592
:10138000F094E094E11CF11C011D111D80E8D82AA5
:101390002AE030E0A101C801B7010E94D90AF82E65
:1013A000F21840C0953729F41D2D1F7E2AE030E049
:1013B0001DC01D2D197F9F3661F0903720F49835A0
:1013C00009F0ADC00FC0903739F0983709F0A7C0C9
:1013D00004C028E030E00AC0106114FD146020E170
:1013E00030E004C014FD166020E132E017FF08C0B1
:1013F000F501608171818281938144E050E008C0F1
:10140000F50180819181BC0180E090E042E050E0F4
:10141000A40EB51EA1010E94D90AF82EF2188FE77A
:10142000D82ED122D6FE0BC05EEFD522F91438F4A7
:10143000D4FE07C0D2FC05C08FEED82202C01F2DFB
:1014400001C0192DD4FE0DC0FE01EF0DF11D8081EC
:10145000803319F499EED92208C01F5FD2FE05C06F
:1014600003C08D2D867809F01F5F0D2DD3FC14C0AD
:10147000D0FE0FC01C1510F09F2C0BC09F2C9C0C95
:10148000911A1C2D06C0B30180E290E00E94AD0AC3
:101490001F5F1C15C0F304C01C1510F4C11A01C055
:1014A000CC2404FF10C0B30180E390E00E94AD0A99
:1014B00002FF1EC001FD03C088E790E002C088E57E
:1014C00090E0B3010CC0802F867891F001FF02C03C
:1014D0008BE201C080E2D7FC8DE2B30190E00E9474
:1014E000AD0A06C0B30180E390E00E94AD0A9A9471
:1014F000F914C0F3FA94F101EF0DF11DB3018081ED
:1015000090E00E94AD0AFF20A9F706C0B30180E277
:1015100090E00E94AD0ACA94CC20C1F741CEF301FD
:1015200066817781CB012B96E2E10C94530BFC0191
:101530000590615070400110D8F7809590958E0FFE
:101540009F1F0895FC016150704001900110D8F771
:10155000809590958E0F9F1F08950F931F93CF93A3
:10156000DF938C01EB018B8181FF1BC082FF0DC0DB
:101570002E813F818C819D812817390764F4E88191
:10158000F9810193F983E88306C0E885F985802F06
:101590000995892B31F48E819F8101969F838E83DB
:1015A00002C00FEF1FEFC801DF91CF911F910F9184
:1015B0000895FA01AA27283051F1203181F1E894E9
:1015C0006F936E7F6E5F7F4F8F4F9F4FAF4FB1E036
:1015D0003ED0B4E03CD0670F781F891F9A1FA11D31
:1015E000680F791F8A1F911DA11D6A0F711D811D32
:1015F000911DA11D20D009F468943F912AE0269FF7
:1016000011243019305D3193DEF6CF010895462F55
:101610004770405D4193B3E00FD0C9F7F6CF462F36
:101620004F70405D4A3318F0495D31FD405241939F
:1016300002D0A9F7EACFB4E0A6959795879577955C
:101640006795BA95C9F700976105710508959B01E3
:10165000AC010A2E06945795479537952795BA956C
:10166000C9F7620F731F841F951FA01D08952F9245
:101670003F924F925F926F927F928F929F92AF9222
:10168000BF92CF92DF92EF92FF920F931F93CF936F
:10169000DF93CDB7DEB7CA1BDB0B0FB6F894DEBF06
:1016A0000FBECDBF09942A88398848885F846E842C
:1016B0007D848C849B84AA84B984C884DF80EE8076
:1016C000FD800C811B81AA81B981CE0FD11D0FB67F
:1016D000F894DEBF0FBECDBFED010895F894FFCFA3
:1016E00053544152540053544F500041444452000B
:1016F00052656164204368616E676520416464726D
:1017000065737320636F6D6D616E640A004F6C6466
:101710003A202564204E65773A2025640A00452545
:101720007325730A00496E76616C6964204D657398
:10173000736167653A2000000000000000000000AF
:101740000000000000000000000000000000000099
:101750000000000000000000000000000000000089
:1017600000000000004572726F72202D20627566C5
:10177000666572206F766572666C6F770A002573F6
:101780002C25640025730A0001030F43684164643B
:10179000722025582025580A0073746172742072D3
:1017A000616E67653A2025640A002000150200007A
:00000001FF
